:1000000021C03BC03AC039C038C037C036C035C047
:1000100034C033C032C031C030C02FC02EC02DC05C
:100020002CC068656C6C6F2E667464692E34342E37
:100030006563686F2E633A20796F752074797065F7
:100040006420000011241FBECFE5D1E0DEBFCDBF8C
:1000500010E0A0E6B0E0EEE8F2E002C005900D92FC
:10006000A036B107D9F710E0A0E6B0E001C01D92BC
:10007000A436B107E1F7ECD008C1C2CFDC01FA0128
:1000800010828C918623E9F78CE18A95F1F788E359
:100090008A95F1F78C91862319F081E0808301C065
:1000A000108288E38A95F1F78C91862319F080817C
:1000B0008260808388E38A95F1F78C91862319F01A
:1000C00080818460808388E38A95F1F78C91862310
:1000D00019F080818860808388E38A95F1F78C919C
:1000E000862319F080818061808388E38A95F1F707
:1000F0008C91862319F080818062808388E38A95C1
:10010000F1F78C91862319F080818064808388E3E5
:100110008A95F1F78C91862319F08081806880831D
:1001200088E38A95F1F78CE18A95F1F70895FC014F
:100130008081962F90958923808388E38A95F1F7B3
:10014000242F332727FD309520FF03C08081862B85
:1001500002C080818923808388E38A95F1F721FF9B
:1001600003C08081862B02C080818923808388E33D
:100170008A95F1F722FF03C08081862B02C080811F
:100180008923808388E38A95F1F723FF03C0808168
:10019000862B02C080818923808388E38A95F1F7CA
:1001A00024FF03C08081862B02C080818923808345
:1001B00088E38A95F1F725FF03C08081862B02C072
:1001C00080818923808388E38A95F1F726FF03C025
:1001D0008081862B02C080818923808388E38A9571
:1001E000F1F747FF04C08081862B808303C08081A4
:1001F0009823908398E3892F8A95F1F78081862B45
:100200008083892F8A95F1F79A95F1F70895EF92F7
:10021000FF921F93CF93DF93EA01EE24FF24FE01A8
:1002200014918BE390E062E0412F81DF0894E11CA0
:10023000F11C2196112399F710926300F09262004D
:10024000E0926100DF91CF911F91FF90EF900895B0
:1002500080E886BD16BCD99AD19A89E390E061E026
:1002600040E650E00BDF8BE390E062E042E250E0DA
:10027000CEDF8BE390E062E04091600058DF8BE3DB
:0E02800090E062E04AE053DFE8CFF894FFCF51
:00000001FF
